:020000040000FA
:04000000803105281E
:040004000034003490
:020008000800EE
:06000A0021007B3099008B
:100010000000000020008C0122008C0123008C01D4
:1000200021008C010C150C168C1620008E0122006C
:100030008E0123008E0121008E018E1423008C146A
:1000400044202000053098009F202000A5012000BA
:10005000F701F001F401F5010630F600F701210087
:10006000161C36200000210016142932CC21210054
:100070008C14CC21CC2121008C10CC2121008C149B
:10008000CC21CC2121008C1021008C1420007F3049
:100090009B0025000C30930025004B30910025007B
:1000A00000309E002000911020009C011C152000B3
:1000B000911CFE3322008E1521008C100800922026
:1000C0007120FC2076080B00AA28B028BC28C7287D
:1000D000D328DC28E828F028F601F601000000000B
:1000E000EE33701C080023000C16210020309E0007
:1000F00021000D309D0022000E14DB21DB21DB21CD
:10010000DB2121009D149D18FE3321001C08F40002
:1001100021009D0123000C1622000E10F436F43647
:10012000F436080070102000111C08001110200087
:10013000A00B080070143D302000A0000800200033
:100140001810200096019701200018143D3020005F
:10015000A00008009F207408043EF500F60A5F28FE
:1001600022000E158E110E12701C5F282000F50B58
:100170005F282000F60A5F282500643091009F2048
:10018000743689368936023EF500F60A5F28220069
:100190000E158E150E12701C5F282000F50B5F28BF
:1001A0002000F60A5F2825004B3091009F2074083C
:1001B000033EF500F60A5F2822000E160E118E117E
:1001C000701C5F282000F50B5F282000F60A5F28CE
:1001D0009F20743609360936033EF500F60A5F287B
:1001E00022008E150E110E12701C5F282000F50BD8
:1001F0005F282000F60A5F28200077080B000F32E6
:1002000010321A3228323A32473257325D32863251
:100210008D329832A032AB32F70100000800F70AA5
:10022000080020000C1908002000F70A2000F60A38
:10023000BA212000A50108000B1D0800BA212000EA
:10024000A50A2508023A031D08002000F70A20002D
:10025000A5010B15080020000C1D0532F70ABA2174
:100260002000A50108000B1D0800BA21A50A2508D9
:10027000323A031D08002000A50126320B1D08009C
:10028000BA212000A50A2508023A031D0800200013
:10029000F70A2000A501080020000C1D3F320B1DAD
:1002A0000800BA212000A50A2508323A031D0800DB
:1002B000A50120000630F7000800BA212000A501A2
:1002C00020000930F700080021008C102500930160
:1002D00021008C1422008C1022000E118E110E129F
:1002E00023000C1222000E1020000C1DFE33C3212F
:1002F000C321C321C321210015138B100B166300EA
:1003000000000B12442023000C1622000E14BA2108
:100310002000A50120000930F7000800F60ABA21E4
:100320002000A50120000930F70008000B1D08007F
:10033000BA212000A50A2508023A031D0800200062
:10034000F70A080020000C1D08002000F70ABA2157
:100350002000A50108000B1D0800BA212000A50AF5
:100360002508023A031D08002000F70A08002000B3
:10037000F70108002100D730950020009C300909C2
:1003800095000B1108002000FA30A200DB21DA21D1
:100390000000A20BC629080020000030A3009C30FA
:1003A000A200DB21DB21DA21D529A30BD129A20B65
:0C03B000D12908000800DC29DD29080024
:020000040001F9
:02000E00E40DFF
:02001000FF1ED1
:00000001FF
